:1000000012C032C031C030C02FC02EC02DC02CC095
:100010002BC02AC029C028C027C026C025C024C0A4
:1000200023C022C021C011241FBECFEDCDBF80E26E
:1000300088BB8FE787BB8CE182BB80E481BB10E08B
:10004000A0E6B0E0E8E0F2E002C005900D92A23632
:10005000B107D9F710E0A2E6B0E001C01D92A236C8
:10006000B107E1F747D0CFC0CBCFC39A0000C39808
:100070000895EF92FF920F931F93082F162FC098A9
:10008000C198F3DFFF24EE2486B3FF0C90E0969531
:100090008795969587958170F82A07FF02C0C09AC8
:1000A00001C0C09817FF02C0C19A01C0C198DDDF2E
:1000B000E39488E0E81619F0000F110FE5CFC0981F
:1000C000C198D3DFD2DF8F2D90E01F910F91FF9069
:1000D000EF90089520E030E0B2990BC086E08A9559
:1000E000F1F72F5F3F4F83E0283E3807A9F71092C2
:1000F000600008950F931F9380E18A95F1F780E3E4
:1001000088BB8DE08A95F1F780E588BB85E08A950C
:10011000F1F7BA9884E68A95F1F780B384FD11C0AF
:100120006CE480E8A6DF64E680E0A3DF6CE680E0B4
:10013000A0DFD0DF6CE480E09CDFCCDF12E60FEDC7
:1001400007C082FD03C011EE0DE502C011EE0DEDFA
:100150006CE480E48EDF6CE2812F8BDF64E680E06C
:1001600088DF6CE680E085DFB5DF6CE480E081DF6E
:10017000B1DF6CE480E47DDF6CE2802F7ADF64E73E
:1001800080E077DF6CE780E074DFA4DF6CE480E080
:1001900070DFA0DF6CE480E46CDF6CE28FEF69DF7E
:1001A00066E680E066DF6EE680E063DF93DF6CE4A6
:1001B00080E05FDF8FDF86E08A95F1F780E388BB20
:1001C00081E08A95F1F780E288BB969A8091600081
:1001D000882351F420E137E289E190E00197F1F7BB
:1001E0002150304029F0F8CF88EA91E60197F1F7E5
:1001F000969885B7806585BF85B7806285BF8895ED
:0802000085B78F7DF8CFFFCF19
:020208000100F3
:00000001FF
